:020000040000FA
:10000000012883128501860183160030810010309B
:1000100085000330860083120F308500FF30860094
:100020001D280F088E0000308C008D008C0B1628C8
:100030008D0B16288E0B1628080019308F00112002
:100040008611061319308F00112086150617061821
:100050001D2806118613851005117D308F00112093
:1000600006158611051585114B308F001120861558
:1000700006128612861705108514FA308F0011209B
:1000800086160613051485104B308F0011200611BB
:100090000616061786130511851506184D282D28F6
:02400E00F23F7F
:00000001FF
